:020000020000FC
:080000000C94EA000C94370097
:040014000C94B10097
:040034000C947C00AC
:040040000C945500C7
:040048000C94880884
:100050000C9459085A9A0E94F8080E85002311F44E
:1000600002E001C003E000936900E89A08950F934D
:100070000FB71F930F9394600F911F910FBF0F91B4
:10008000189507E005BBF4BC05E005BD0895A1E3A4
:10009000B1E0AAA7BBA700E006BD01E000936E0097
:1000A000089500E000936E0008950F9378940FB7C1
:1000B0000F93BF93AF93AAA5BBA5AE19BF09AAA77B
:1000C000BBA739F4EEDF0CA5002319F498600FEFFD
:1000D0000AA3AF91BF910F910FBF0F91189504E044
:1000E000009381000AEF009385000AEE00938400DC
:1000F00001E000936F0008950F930AEE00938400CF
:100100000AEF0093850078940FB71F930F930F8128
:100110000A9511F4906808850F8309890A9511F4EE
:1001200090640FE0098B0DA500FF08C00EA50A958D
:100130000EA721F40E7F0DA706D022D00F911F919C
:100140000FBF0F91189510E810936D0014E01093F5
:100150006800089510E010936D0010E0109368009F
:1001600008950F930FB71F930F93F4DF13E01EA7AB
:100170001DA511601DA70F911F910FBF0F9118951D
:100180001F930F934F9B09C08CDF0AA1002339F006
:100190000F3F29F09260FAA202C0EAA278DF0F9125
:1001A0001F910895A89504B7077F04BF00916000D0
:1001B000086100936000F09260000895F894A8959B
:1001C000009160000861009360000AE00093600005
:1001D00078940895589A599AE5DFCEE1D1E0FF244A
:1001E000EE24E3949927BB24CC24FDA6FEA6FCA60E
:1001F000FB86FC8AFAA2FBA20FEF0E8BFF8AFDA200
:10020000FEA2FA8AFB8AF9A6F8A6EAE1F3E1E093F6
:100210000001F0930101FFA2EAEAF4E1E093020198
:10022000F0930301EEE6FBE1E0931A01F0931B016A
:10023000E6E0F6E1E0930A01F0930B010CE308839A
:100240000EE30F8308870FE0098B36D60E8789D619
:1002500027D60D8705E0088FF98E25D60CA300233D
:1002600011F00FEF098F25D60F8729D609A301ECCE
:100270000093640006DF33DFBDD6E1D7FED6D4D2CB
:10028000DCD261DF25D60F3F69F48827B9D48827EF
:10029000C1D48827C7D481E0CDD481E0D3D48827C6
:1002A000D9D4F0D5FAD50FA3002331F0E6E0F6E17A
:1002B000E0930201F0930301F9D50C87002311F4B8
:1002C0000FE001C007E00A87098743D4CFD18980B6
:1002D00031D05BD409810815D9F30A95098354D12B
:1002E000B9DE7894F3D2BCD4F1D2DDD623D090FD20
:1002F00014D3FCCF0F921F920F931F932F933F9312
:100300004F936F938F93BF93AF93FF93EF935F934D
:100310007F9310D07F915F91EF91FF91AF91BF914B
:100320008F916F914F913F912F911F910F911F903E
:100330000F900895B9D091FF02C09D7F3FDF92FFDB
:1003400011C00EA1002311F41FD101C05CD11CA566
:1003500010FF05C011FFECD512FDF1D501C0E8D5A5
:100360009B7F098197FF08C0D7D50EA1002311F408
:100370000BD101C048D19F7796FF6AC00A8900FF60
:1003800013C00B8900FD07C0E4E3F5E1E0930A0127
:10039000F0930B0106C0E6E0F6E1E0930A01F0936A
:1003A0000B01019503950B8B0C890023A1F00D899E
:1003B00000FD07C0E0EAF5E1E0930C01F0930D01C8
:1003C00006C0E6E0F6E1E0930C01F0930D01019523
:1003D00003950D8B16C00E890E1599F40F8900FD3B
:1003E00007C0E6E8F5E1E0930C01F0930D0106C0CB
:1003F000E6E0F6E1E0930C01F0930D010195039521
:100400000F8B09A5002319F10B85002301F508A521
:1004100000FD10C0EAE1F3E1E0930001F093010177
:100420000FA0002089F4EAEAF4E1E0930201F093DE
:1004300003010AC0E6E0F6E1E0930001F093010158
:10044000E0930201F09303010195039508A79F7BB8
:1004500094FF24C0088D0A9511F471D505E0088F2A
:1004600009A1002311F001E034D30A89002341F0EF
:10047000FA8AFB8AE6E0F6E1E0930A01F0930B01C9
:100480009F7E95FF0BC019A10D8510230CA1102391
:1004900021F00B81043009F4EA8A9F7D93FF03C0A9
:1004A000977F0E94041408951127A0E0B1E0A10FE6
:1004B000BF1DA10FBF1DED91FD91139509850395FA
:1004C00010170CF011C05D9A85918823E1F36591B6
:1004D00045914423C1F34F3F41F325912F934F930F
:1004E00005D08F916F91F4CF5D9A0895772790D5BD
:1004F0005D9991D50FEFA82FA41B10F4AA95A02702
:10050000B62FB21B10F4BA95B0270A2F0B1B50F46C
:100510007860862768278627422724274227AB272B
:10052000BA27AB277D7F042F081B08F472607B7FFE
:10053000022F061B08F4746055275D9873FD02C0F6
:100540006AD501C081D58417C9F05B0F08F47F7E9E
:1005500074FD0EC00A2F0894050B08F009C07F7EB9
:100560005A1B08F4706172FD02C0639501C06A9560
:1005700071FD02C08395E2CF8A95E0CF73FF03C07F
:1005800086276827862708950F921F921F930F933F
:100590003F932F93FF93EF934AD108850F831981DF
:1005A000139519831C3341F00BA1002311F0FBA21A
:1005B0001EC083D0ECD01EC090611E85112319F49B
:1005C000EFD2C7D214C0F9821A8113951A831C3353
:1005D0004CF09062FA821B8113951B83183114F042
:1005E000FB8205C01DA1112311F4F7D2B2D243D072
:1005F00070D0F8D0EF91FF912F913F910F911F9103
:100600001F900F9008951E85112329F110D10885A0
:100610000F8319811A9519831F3F41F00BA1002305
:1006200011F0FBA215C049D0B2D015C01BE319834D
:1006300090611A811A951A831F3F51F41BE31A83A4
:1006400090621B811A951B831F3F11F417E11B83D6
:1006500012D03FD0C7D008951DA10EA1102B29F4B0
:100660009FD209D036D0BED00895089599D203D034
:1006700030D0B8D0089521D0E6E3F7E10A8129E02F
:10068000029FE00DF11DE0930601F0930701E2E502
:10069000F9E10A811CE07AD40F930B8177D4022F01
:1006A00025E0029F1F91100D29E0129FE00DF11D22
:1006B000E0930801F09309010895EAE0F6E1098169
:1006C00015E0019FE00DF11DE0930401F093050199
:1006D00008955DD00A811AE059D4000F0F840020DC
:1006E00019F0EAE1FEE102C0E4ECF1E2E00FFF1DE7
:1006F00005911491000F111F00931401109315011F
:10070000022F000F0F84002019F0ECE3FDE102C07E
:10071000E6EEF0E2E00FFF1D05911491000F111FAE
:1007200000931201109313010B810F8400FC05C08C
:10073000E2E5F3E2E00FFF1D04911AE027D4000F79
:100740000F84002019F0E8E6FFE102C0E2E1F3E2E5
:10075000E00FFF1D05911491000F111F0093180168
:1007600010931901022F000F0F84002019F0EAE8FE
:10077000FEE102C0E4E3F2E2E00FFF1D05911491F7
:10078000000F111F0093160110931701089509819E
:100790001AE0FCD3000F0F84002019F0ECECFCE110
:1007A00002C0E6E7F0E2E00FFF1D05911491000F93
:1007B000111F0093100110931101022F000F0F84DD
:1007C000002019F0EEEEFBE102C0E8E9FFE1E00FE6
:1007D000FF1D05911491000F111F00930E0110933E
:1007E0000F0108950F85002391F4EAE9FBE1E093FE
:1007F0001A01F0931B01E2EDFBE10B810C3014F0C8
:10080000EEEDFBE1E0931C01F0931D010CC0EEE660
:10081000FBE1E0931A01F0931B01E6E0F6E1E093BF
:100820001C01F0931D010895569A5E9808950D8558
:1008300000FF4E9A08955E98089557985F9A08951C
:100840000F9309818EE1080F0C330CF00C53CAD4BE
:10085000882329F44FDD8981081729F0F8CF80D447
:10086000C2D30F91089588E50F9108958F93BED458
:10087000882311F43FDDFBCF8F9169D40895B6D45E
:10088000882311F437DDFBCF86D408958F93AED43F
:10089000882311F42FDDFBCF8F9118D00895A6D4B3
:1008A000882311F427DDFBCF86D408950F939ED4BF
:1008B000882311F41FDDFBCF0F91002319F0EAE428
:1008C000F5E269C4EEE4F5E266C40895E6E4F5E213
:1008D00062C412E0B9D48F7764D3839583958C3347
:1008E0000CF08C53082E00E405DD0A950023E1F797
:1008F00012E0AAD48F7755D30816A9F70895E9DF37
:10090000E8DF0895FCDFFBDF0895B9DFBFDFE1DF3B
:100910000895B5DFBBDFF3DF08958F931F930F9327
:100920003F932F93BF93AF93FF93EF930F921F9239
:1009300017D459D3883509F08BC0E0EAF3E29FDF82
:100940007FDF94DFA3DF8435C9F1843409F468C004
:10095000833509F463C08C3411F427D279C0813413
:1009600011F4F3D175C0863511F456D271C08334B9
:1009700011F491D16DC08E3411F404D269C0803568
:1009800011F423D265C0823411F42DD261C08135B7
:1009900011F4B2D15DC0823511F4C6D159C086348C
:1009A00011F444D255C0873511F4ACDF51C08834FE
:1009B00011F4E8D24DC0883569F1BFCFEAECF3E21B
:1009C0005EDF54D030F12ED161DFE2EEF3E257DF8B
:1009D0004DD0F8F01FD15ADFEAEFF3E250DF46D0F6
:1009E000C0F00E85002351F48F9389818F935CDDD5
:1009F0008F91CBD009810817C9F38F9101D1EBA258
:100A000009810A950983C0DD9B7740DF002761D00B
:100A100004C02CDEECE1F5E232DF1AC021D118C0AF
:100A2000E2E1F4E22CDF22D0A8F314D12FDFEAE2D6
:100A3000F4E225DF1BD070F305D128DFE2E4F4E215
:100A40001EDF14D038F3F6D021DF002742D000C0DB
:100A50001DDFEBA21F900F90AF91BF91EF91FF911F
:100A60002F913F910F911F918F910895E9DEFEDE46
:100A7000883511F4089408950DD0C0F3082FE0DEF6
:100A8000F5DE8835B9F306D0D0F31AE0019F800D6A
:100A900088940895803328F08A3318F4805388941A
:100AA000089508940895EAE7F3E2E9DE82E3DEDEE2
:100AB0008EE2DCDE84E3DADEE9DE089582D28F9313
:100AC00082958F7086D28D938F918F7082D28D9305
:100AD00008958CD3882311F40DDCFBCFFF93EF93A3
:100AE000BF93AF930F93ADE4B1E08C81E7DF8DE26C
:100AF0008D938D81E2E5F5E28A95880F880FE80FE6
:100B0000FF1D85918D9385918D9385918D938DE2B8
:100B10008D9382E38D9380E38D938E81CFDF80E28E
:100B20008D938B81CBDF8AE38D938A81C7DF8AE344
:100B30008D938981C3DF0F91002321F08DE08D9388
:100B40008AE08D93FD9237D3AF91BF91EF91FF91E2
:100B500008950F938F9315E077D38F7322D280324D
:100B60000CF08E2D8C8317E06FD38F711AD28D30DD
:100B70000CF08E2D8D8318E067D313D283360CF0E2
:100B800088278E838F910F9108958F9312E05CD305
:100B90008F7707D28C330CF0882789838F91089543
:100BA0008F9312E051D387FDA2D18F77FAD18C3386
:100BB0000CF08827898313E047D38F77F2D18C33E9
:100BC0000CF088278A8314E03FD38F73EAD18831F1
:100BD0000CF088278B838F9108958CA5882379F456
:100BE0008981EFD112E0082F48D38A81EAD113E03E
:100BF000082F43D38B81E5D114E0082F3ED308950D
:100C00008F93082F0C3320F48983DBD112E035D386
:100C10008F910895082F0C3320F48A83D2D113E0EA
:100C20002CD30895082F083120F48B83CAD114E007
:100C300024D30895082F003220F48C83C2D115E00C
:100C40001CD30895082F0C3020F48D83BAD117E0FF
:100C500014D30895082F8E83B4D118E00ED30895CD
:100C600022DF002736DF80E201DE82E50E850023E9
:100C700009F081E4FBDD0D85002311F48CE4F6DD41
:100C80000CA1002311F482E4F1DD09A1002311F08D
:100C900086E5ECDD08952F93EAE5F4E2F0DD0B85BF
:100CA000002339F0BFD2002722271A85EAE1F3E1B9
:100CB00009C015D0B3D20E2D2FEFBB24CC2411E0E8
:100CC000ECEEF5E11987E0930001F09301011CA11E
:100CD000112309F4298F0B87E9DD2F9108950DA1C8
:100CE000002321F01EE318871F83FDA20EA100231D
:100CF00009F0FEA2B1DC08950E8500FD04C0EAED06
:100D0000F4E2BDDD10C0E0ECF4E2B9DD0DA100239A
:100D100019F01EE3002702C012E00E2D18871F8372
:100D20000DA3C4DD99DC08950E8500FD04C0EAED35
:100D3000F4E2A5DD09C0ECECF4E2A1DD0EA1019521
:100D400003950EA3B3DD88DC0895EAE9F4E297DDAC
:100D50000E85002349F0C3DF0027E6E0F6E1E093CB
:100D60000C01F0930D0107C00395EAE7F5E1E0936C
:100D70000C01F0930D010E877CD098DD0CA500FFCF
:100D80001DDA0895E0E7F4E27ADD0C85002319F01E
:100D900000271FE002C0039517E00C8719871A8708
:100DA00065D00195039582DD0895E2E8F4E267DD00
:100DB0000D85002311F0002702C003953CDD0D874F
:100DC0004FD00195039572DD0895E2E9F4E257DD15
:100DD0000F85019503950F874FD00195039566DD2B
:100DE00001DD77DC0895ECEAF4E249DD0CA1019520
:100DF00003950CA30F9337D00195039557DD0F9101
:100E00001B85112341F4002329F00FEF098FBB2428
:100E1000CC2401C0F98E0895E8E8F4E230DD09A1A0
:100E20000195039509A32BD041DD0895E8E0F5E293
:100E300026DD0FA1002321F00027EAEAF4E103C038
:100E40000395E6E0F6E1E0930201F09303010FA3BE
:100E500004D0019503952ADD0895A7E0B0E016C0FF
:100E6000A0E0B0E013C0A6E0B0E010C0A3E0B0E0A6
:100E70000DC0A2E0B0E00AC0A4E0B0E007C0A1E06D
:100E8000B0E004C0A5E0B0E001E000C00CA4002088
:100E900019F400BD16E021D00895A7E0B0E012C01B
:100EA000A0E0B0E00FC0A6E0B0E00CC0A3E0B0E06E
:100EB00009C0A4E0B0E006C0A2E0B0E003C0A1E039
:100EC000B0E000C011E009D00F3F09F400270895F9
:100ED000A5E0B0E011E001D00895A1BDB2BD11962A
:100EE00011FDFA9A1FBBF999FECF00B508950E893E
:100EF0000F3F41F4EE8AEF8AE6E8F5E1E0930C015A
:100F0000F0930D0108950FEF0E8BFF8AE6E0F6E1F6
:100F1000E0930C01F0930D010DA100FD0895EC8A02
:100F2000ED8AE0EAF5E1E0930C01F0930D010895FC
:100F30000C8900FF0895FC8AFD8A13D00895098D5D
:100F40000F3F71F0FF93EF93EAE6F3E2039507702A
:100F5000098F000FE00FFF1DB590C490EF91FF9136
:100F600008950E85002339F4E6E0F6E1E0930C01E4
:100F7000F0930D0106C0EAE7F5E1E0930C01F09370
:100F80000D010895E2E8F5E27ADC0895222738E0C1
:100F9000000F221F211710F00395211B3A95C1F76E
:100FA00008950F921F920F938F9382958F700AE08E
:100FB000809F002D8F918F70800F0F911F900F9049
:100FC0000895082F1AE0E2DF07700295022B802FA8
:100FD0000895FF93EF93E2E4F3E2E80FFF1D84919D
:100FE000EF91FF910895813624F08B3710F400E2E1
:100FF000801B0895209A219A229A239A389A399A26
:101000003A9A3B9A539A549A559A5D9A5C9A0895E3
:1010100038B1307F08958F938B0D5B98082F8F70B8
:10102000832B88B9029505B9862F81958C0D082FE1
:101030008F70832B02955C985C9A5B9A88B905B98E
:101040005C985C9A8F9108956F936B0D5B98062F57
:101050006F70632B68B9029505B9682F61956C0DA7
:10106000062F6F70632B02955C985C9A5B9A68B947
:1010700005B95C985C9A6F91089510E41093C400D0
:10108000F092C500F092C00018E41093C10016E081
:101090001093C200F8A2EA8EFE8EFF8EFB8EFC8EAD
:1010A0001FEF1D8F08951091C10010691093C100AA
:1010B0000895AFB60F931F93FF93EF930D8D0F3FDE
:1010C00079F00395EDE4F1E0E00FFF1D10811123AD
:1010D00019F40FEFEA8E02C01093C6000D8F12C0F4
:1010E000EB8DFC8D0E2F0F2B39F0EF5FFF4F14911E
:1010F000112321F4FB8EFC8EEA8E04C01093C600EF
:10110000EB8FFC8FEF91FF911F910F91AFBE189560
:10111000AFB60F931F932F933F93FF93EF932091BD
:10112000C6000E8D302F03950F701F8D011739F0FB
:101130000E8FEDECF1E0E30FFF1D20839160EF9146
:10114000FF913F912F911F910F91AFBE18950F9373
:101150000A8D0023E9F3FA8E8093C6000F9108955B
:1011600090FFFECF0F931F93FF93EF931E8D0F8D74
:101170008827011751F0EDECF1E0E00FFF1D8081B1
:1011800003950F700F8F011709F49E7FEF91FF9168
:101190001F910F9108950F93FF93EF930A8D0023F2
:1011A000E9F3FA8EEB8FFC8F04910093C600EF9168
:1011B000FF910F9108950F93FF93EF930A8D0023F2
:1011C000E9F3FA8EFD8EEDE4F1E00081002321F4D5
:1011D0000FEF0D8FEA8E02C00093C600EF91FF91D2
:1011E0000F910895882790FD839508958A8D08951D
:1011F0001F930F9317D01FE000E43FD01EE001E8DB
:101200003CD011E001E139D00F911F9108951FE00A
:1012100000E433D011E001E130D008951DE000E892
:101220002CD008951DE0002728D00895000000006C
:1012300000000000000000000000000008953C9A3B
:101240003D9A449A459A08955ED0F0DF02EA36D07E
:10125000EDDF2AD0C8F3012F31D0E8DF25D0A0F38D
:101260004CD051D003EA2AD0E1DF1ED068F333D04E
:10127000449A459A42D0802F089545D0D7DF0F93E6
:1012800002EA1CD0D3DF10D00F91B8F30F93012FD7
:1012900015D00AD00F9188F30F9310D005D00F917D
:1012A00060F300002AD008953C98449A0894459A27
:1012B000BDDF349B889445983C9A08953F9338E06D
:1012C000449A000F08F04498459AB0DF45983A9543
:1012D000B9F73F9108953F933C98449A00E038E075
:1012E000459A0894A3DF349B8894001F45989EDF9D
:1012F0003A95B1F73C9A3F9108954498459A000079
:101300000000449A0895449A459A000000004498C9
:10131000000000004598000008957A157A270080A3
:1013200018831589158C188C1B80278C270086DC68
:1013300083D97DD97ADC7AE87DEB83EB86E886E594
:1013400083E27DE27AE500E07AE377E977EC7AEC14
:101350007DE980EC83EC86E989E389E08600E3801F
:10136000E980001F7D1C801C801680137D137A1677
:10137000771C771F7A1F861C8916891386008002C6
:10138000800E008D028C07009A04990900A608A51A
:101390000C00B30CB11100BF12BA1B00CA1AC71E51
:1013A00000D422D02600DD2BD92F00E535E138000E
:1013B000ED41E44600F34CEE4E00F759F35A00FBC2
:1013C00065F66600FD72F87300FD80F18000FD8D0A
:1013D000F88C00FB9AF69900F7A6F3A500F3B3EE9C
:1013E000B100EDBFE4BA00E5CAE1C700DDD4D9D051
:1013F00000D4DDD0D900CAE5C7E100BFEDBAE400F2
:10140000B3F3B1EE00A6F7A5F3009AFB99F6008DB1
:10141000FD8CF8007FFD7FF10072FD73F80065FB25
:1014200066F60059F75AF3004CF34EEE0041ED46D4
:10143000E40035E538E1002BDD2FD90022D426D099
:10144000001ACA1EC70012BE1BB9000CB311B100AE
:1014500008A60CA500049A099900028D078C0002C9
:101460007F0E7F0002720773000465096600085949
:101470000C5A000C4C114E0012411B46001A351E2E
:101480003800222B262F002B222F2600351A381E3B
:10149000004012451B004C0C4E110059085A0C001C
:1014A000650466090072027307FFB51CB52E0000C3
:1014B000D245D542DB42DE45DE48D254DE54000040
:1014C000E0B4D4B4DDABDDBD0000B8CFACCFACD858
:1014D000B5D8B8DBB8DEB5E1AFE1ACDE000047CF90
:1014E00053CF53D250D54DDB4DE1000022B41FB194
:1014F0001FAE22AB28AB2BAE2BB128B422B41FB742
:101500001FBA22BD28BD2BBA2BB728B40000214238
:101510002154000027452A4230423345335130548C
:101520002A54275127450000491C492E0000531C0E
:10153000532EFF00B25CB25ABA5ABA66B266B264AF
:1015400000BE66BE62C462C466BE6600C466C45A9B
:1015500000C966C95ACD5ACF5CCF60CD62C962005E
:10156000CD62CF66FF007E467E3A823A843C84405C
:1015700082427E420082428446FF7C46803A844614
:101580000082427E42FF7C467C3A823A843C843E22
:1015900082407C4082408442844482467C46FF00F4
:1015A0007E467E3A823A843C843E82407E40FF0002
:1015B000A764AD64AF66AF6EAD70A770A76400BBE3
:1015C00064B364B370BB7000B96AB36A00BE70BE26
:1015D00064C268C664C67000C966CB64CF64D16655
:1015E000D16ECF70CB70C96EC966FF0001FE0101DC
:1015F000FE01FEFE01FEFE010101FEFE01FE0101F3
:10160000FE01FEFEFF000101FF0080148080FF8BC1
:10161000148080FF96168080FFA1198080FFAB1D8B
:101620008080FFB6228080FFBF288080FFC82F8087
:1016300080FFD0378080FFD7408080FFDD4A8080E8
:10164000FFE2548080FFE65E8080FFE9698080FFD2
:10165000EB748080FFEB808080FFEB8B8080FFE964
:10166000968080FFE6A18080FFE2AB8080FFDDB640
:101670008080FFD7BF8080FFD0C88080FFC8D08027
:1016800080FFBFD78080FFB6DD8080FFABE2808027
:10169000FFA1E68080FF96E98080FF8BEB8080FFD2
:1016A0007FEB8080FF74EB8080FF69E98080FF5EC4
:1016B000E68080FF54E28080FF4ADD8080FF40D7D3
:1016C0008080FF37D08080FF2FC88080FF28BF80B8
:1016D00080FF22B58080FF1DAB8080FF19A1808034
:1016E000FF16968080FF148B8080FF147F8080FF20
:1016F00014748080FF16698080FF195E8080FF1D52
:10170000548080FF224A8080FF28408080FF2F374E
:101710008080FF372F8080FF40288080FF49228013
:1017200080FF541D8080FF5E198080FF69168080D5
:10173000FF74148080FF8280801A7E808280FF8107
:10174000808A1A7E7F8180FF8180951C7E7F8180C8
:10175000FF81809F1E7E7F8180FF8180A9227E7F06
:101760008180FF8181B3277E7E8181FF8181BB2DB6
:101770007E7E8181FF8181C4347E7E8181FF818173
:10178000CB3B7E7E8181FF8181D2447E7E8181FF41
:101790008081D84D7F7E8081FF8081DD567F7E8075
:1017A00081FF8081E1607F7E8081FF8081E36A7FAD
:1017B0007E8081FF8081E5757F7E8081FF7F82E56D
:1017C00080807E7F82FF7F81E58A807E7F81FF7FB0
:1017D00081E395807E7F81FF7F81E19F807E7F8195
:1017E000FF7F81DDA9807E7F81FF7E81D8B3817EEE
:1017F0007E81FF7E81D2BB817E7E81FF7E81CBC4D4
:10180000817E7E81FF7E81C4CB817E7E81FF7E8151
:10181000BBD2817E7E81FF7E81B3D8817E7E81FFB7
:101820007E80A9DD817F7E80FF7E809FE1817F7E3B
:1018300080FF7E8095E3817F7E80FF7E808AE581C8
:101840007F7E80FF7E7F7FE582807E7FFF7E7F754B
:10185000E581807E7FFF7E7F6AE381807E7FFF7EE1
:101860007F60E181807E7FFF7E7F56DD81807E7F8D
:10187000FF7E7F4DD881807E7FFF7E7E44D2818136
:101880007E7EFF7E7E3BCB81817E7EFF7E7E34C46A
:1018900081817E7EFF7E7E2DBB81817E7EFF7F7E6D
:1018A00027B280817F7EFF7F7E22A980817F7EFF9D
:1018B0007F7E1E9F80817F7EFF7F7E1C9580817F43
:1018C0007EFF7F7E1A8A80817F7EFF807E1A7F7FE7
:1018D00082807EFF807E1A757F81807EFF807E1CE5
:1018E0006A7F81807EFF807E1E607F81807EFF8098
:1018F0007E22567F81807EFF807E274D7F81807E85
:10190000FF817E2D447E81817EFF817E343B7E81FE
:10191000817EFF817E3B347E81817EFF817E442DEE
:101920007E81817EFF817E4C277E81817EFF817F4B
:1019300056227E80817FFF817F601E7E80817FFFB7
:10194000817F6A1C7E80817FFF817F751A7E808106
:101950007FFF828080447E808280FF818086447EFB
:101960007F8180FF81808C457E7F8180FF81809296
:10197000467E7F8180FF818098497E7F8180FF81C4
:10198000819E4C7E7E8181FF8181A34F7E7E8181FD
:10199000FF8181A8537E7E8181FF8181AC577E7E4D
:1019A0008181FF8181B05C7E7E8181FF8081B36215
:1019B0007F7E8081FF8081B6677F7E8081FF80810E
:1019C000B96D7F7E8081FF8081BA737F7E8081FFC9
:1019D0008081BB797F7E8081FF7F82BB80807E7F1C
:1019E00082FF7F81BB86807E7F81FF7F81BA8C8072
:1019F0007E7F81FF7F81B992807E7F81FF7F81B66C
:101A000098807E7F81FF7E81B39E817E7E81FF7E76
:101A100081B0A3817E7E81FF7E81ACA8817E7E81A4
:101A2000FF7E81A8AC817E7E81FF7E81A3B0817E16
:101A30007E81FF7E819EB3817E7E81FF7E8098B60F
:101A4000817F7E80FF7E8092B9817F7E80FF7E8055
:101A50008CBA817F7E80FF7E8086BB817F7E80FF07
:101A60007E7F7FBB82807E7FFF7E7F79BB81807E91
:101A70007FFF7E7F73BA81807E7FFF7E7F6DB9811D
:101A8000807E7FFF7E7F67B681807E7FFF7E7F6264
:101A9000B381807E7FFF7E7E5CB081817E7EFF7E13
:101AA0007E57AC81817E7EFF7E7E53A881817E7EC3
:101AB000FF7E7E4FA381817E7EFF7F7E4C9D808155
:101AC0007F7EFF7F7E499880817F7EFF7F7E46926A
:101AD00080817F7EFF7F7E458C80817F7EFF7F7E41
:101AE000448680817F7EFF807E447F7F82807EFF70
:101AF000807E44797F81807EFF807E45737F8180F8
:101B00007EFF807E466D7F81807EFF807E49677F7D
:101B100081807EFF807E4C627F81807EFF817E4F50
:101B20005C7E81817EFF817E53577E81817EFF8135
:101B30007E57537E81817EFF817E5C4F7E81817ED8
:101B4000FF817E614C7E81817EFF817F67497E803F
:101B5000817FFF817F6D467E80817FFF817F73451E
:101B60007E80817FFF817F79447E80817FFF6EADA3
:101B70006EAB70AB70AD6EAD006EB16EB370B37026
:101B8000B16EB1008FAD8FAB91AB91AD8FAD008FCA
:101B9000B18FB391B391B18FB1FF62AD62AB64AB62
:101BA00064AD62AD0062B162B364B364B162B100AE
:101BB00082AD82AB84AB84AD82AD0082B182B3844E
:101BC000B384B182B100AEB5AEA9B2ADB6A9B6B517
:101BD000FF00A2B5A6A9AAB500A8B1A4B1FFA4B5FB
:101BE000A4A9A8A9AAABAAADA8AFA4AFFF00010EF3
:101BF0000B0E0E0E160E240E290E330E400E470E3F
:101C0000580EA2ABA4A9A8A9AAABAAB3A8B5A4B51B
:101C1000A2B3A2ABFF00A6A9A6B5FF00A2ABA4A9E0
:101C2000A8A9AAABAAADA2B5AAB5FF00A2ABA4A968
:101C3000A8A9AAABAAADA8AFAAB1AAB3A8B5A4B5E2
:101C4000A2B300A4AFA8AFFFAAAFA2AFA8A9A8B53E
:101C5000FF00AAA9A2A9A2AFA8AFAAB1AAB3A8B52A
:101C6000A4B5A2B3FF00AAABA8A9A4A9A2ABA2B332
:101C7000A4B5A8B5AAB3AAB1A8AFA4AFA2B1FF00FA
:101C8000A2A9AAA9AAABA8ADA6B1A6B5FF00A4AF08
:101C9000A2ADA2ABA4A9A8A9AAABAAADA8AFA4AFB4
:101CA000A2B1A2B3A4B5A8B5AAB3AAB1A8AFFF00C8
:101CB000AAADA8AFA8AFA4AFA2ADA2ABA4A9A8A992
:101CC000AAABAAB3A8B5A4B5A2B3FF006C0E760E5A
:101CD000790E810E8F0E940E96AB98A99CA99EAB9F
:101CE0009EB39CB598B596B396ABFF009AA99AB5EA
:101CF000FF0096AB98A99CA99EAB9EAD96B59EB5EC
:101D0000FF0096AB98A99CA99EAB9EAD9CAF9EB1DF
:101D10009EB39CB598B596B30098AF9CAFFF9EAFAD
:101D200096AF9CA99CB5FF009EA996A996AF9CAFC3
:101D30009EB19EB39CB598B596B3FF00A80EB20EA7
:101D4000B50EBD0ECB0ED00EDA0EE70EEE0EFF0E68
:101D500082AB84A988A98AAB8AB388B584B582B3DB
:101D600082ABFF0086A986B5FF0082AB84A988A953
:101D70008AAB8AAD82B58AB5FF0082AB84A988A9F7
:101D80008AAB8AAD88AF8AB18AB388B584B582B38D
:101D90000084AF88AFFF8AAF82AF88A988B5FF0003
:101DA0008AA982A982AF88AF8AB18AB388B584B57F
:101DB00082B3FF008AAB88A984A982AB82B384B5C1
:101DC00088B58AB38AB188AF84AF82B1FF0082A997
:101DD0008AA98AAB88AD86B186B5FF0084AF82AD93
:101DE00082AB84A988A98AAB8AAD88AF84AF82B15F
:101DF00082B384B588B58AB38AB188AFFF008AAD53
:101E000088AF88AF84AF82AD82AB84A988A98AAB42
:101E10008AB388B584B582B3FF00130F1D0F200F5E
:101E2000280F360F3B0F76AB78A97CA97EAB7EB32B
:101E30007CB578B576B376ABFF007AA97AB5FF00AA
:101E400076AB78A97CA97EAB7EAD76B57EB5FF007A
:101E500076AB78A97CA97EAB7EAD7CAF7EB17EB33C
:101E60007CB578B576B30078AF7CAFFF7EAF76AF48
:101E70007CA97CB5FF007EA976A976AF7CAF7EB148
:101E80007EB37CB578B576B3FF004F0F590F5C0F6A
:101E9000640F720F770F810F8E0F950FA60F62AB35
:101EA00064A968A96AAB6AB368B564B562B362AB8A
:101EB000FF0066A966B5FF0062AB64A968A96AABBA
:101EC0006AAD62B56AB5FF0062AB64A968A96AAB86
:101ED0006AAD68AF6AB16AB368B564B562B30064ED
:101EE000AF68AFFF6AAF62AF68A968B5FF006AA9C3
:101EF00062A962AF68AF6AB16AB368B564B562B32C
:101F0000FF006AAB68A964A962AB62B364B568B547
:101F10006AB36AB168AF64AF62B1FF0062A96AA92F
:101F20006AAB68AD66B166B5FF0064AF62AD62AB27
:101F300064A968A96AAB6AAD68AF64AF62B162B305
:101F400064B568B56AB36AB168AFFF006AAD68AFDF
:101F500068AF64AF62AD62AB64A968A96AAB6AB3EB
:101F600068B564B562B3FF00B70FC10FC40F55ABBE
:101F700057A95BA95DAB5DB35BB557B555B355AB21
:101F8000FF0059A959B5FF0055AB57A95BA95DAB37
:101F90005DAD55B55DB5FF00D60FE00FE30FEB0F5C
:101FA000F90FFE0F081015101C102D1096AB98A9F4
:101FB0009CA99EAB9EB39CB598B596B396ABFF001B
:101FC0009AA99AB5FF0096AB98A99CA99EAB9EAD25
:101FD00096B59EB5FF0096AB98A99CA99EAB9EAD09
:101FE0009CAF9EB19EB39CB598B596B30098AF9C3C
:101FF000AFFF9EAF96AF9CA99CB5FF009EA996A986
:1020000096AF9CAF9EB19EB39CB598B596B3FF00BA
:102010009EAB9CA998A996AB96B398B59CB59EB378
:102020009EB19CAF98AF96B1FF0096A99EA99EABBA
:102030009CAD9AB19AB5FF0098AF96AD96AB98A9B2
:102040009CA99EAB9EAD9CAF98AF96B196B398B548
:102050009CB59EB39EB19CAFFF009EAD9CAF9CAF64
:1020600098AF96AD96AB98A99CA99EAB9EB39CB534
:1020700098B596B3FF0041104B104E1056106410E7
:1020800069108AAB8CA990A992AB92B390B58CB52C
:102090008AB38AABFF008EA98EB5FF008AAB8CA9EC
:1020A00090A992AB92AD8AB592B5FF008AAB8CA98C
:1020B00090A992AB92AD90AF92B192B390B58CB51E
:1020C0008AB3008CAF90AFFF92AF8AAF90A990B562
:1020D000FF0092A98AA98AAF90AF92B192B390B54E
:1020E0008CB58AB3FF007D1087108A109210A01063
:1020F000A510AF10BC10C310D41076AB78A97CA982
:102100007EAB7EB37CB578B576B376ABFF007AA9AB
:102110007AB5FF0076AB78A97CA97EAB7EAD76B5AB
:102120007EB5FF0076AB78A97CA97EAB7EAD7CAF97
:102130007EB17EB37CB578B576B30078AF7CAFFF67
:102140007EAF76AF7CA97CB5FF007EA976A976AF7D
:102150007CAF7EB17EB37CB578B576B3FF007EAB45
:102160007CA978A976AB76B378B57CB57EB37EB121
:102170007CAF78AF76B1FF0076A97EA97EAB7CAD4F
:102180007AB17AB5FF0078AF76AD76AB78A97CA945
:102190007EAB7EAD7CAF78AF76B176B378B57CB5EB
:1021A0007EB37EB17CAFFF007EAD7CAF7CAF78AFFD
:1021B00076AD76AB78A97CA97EAB7EB37CB578B5DD
:1021C00076B3FF00E810F210F510FD100B1110119E
:1021D0006AAB6CA970A972AB72B370B56CB56AB317
:1021E0006AABFF006EA96EB5FF006AAB6CA970A95F
:1021F00072AB72AD6AB572B5FF006AAB6CA970A91B
:1022000072AB72AD70AF72B172B370B56CB56AB3C8
:10221000006CAF70AFFF72AF6AAF70A970B5FF000E
:1022200072A96AA96AAF70AF72B172B370B56CB5BA
:102230006AB3FF0024112E113111391147114C11CD
:10224000561163116A117B1156AB58A95CA95EAB9C
:102250005EB35CB558B556B356ABFF005AA95AB534
:10226000FF0056AB58A95CA95EAB5EAD56B55EB536
:10227000FF0056AB58A95CA95EAB5EAD5CAF5EB12A
:102280005EB35CB558B556B30058AF5CAFFF5EAFF8
:1022900056AF5CA95CB5FF005EA956A956AF5CAF0E
:1022A0005EB15EB35CB558B556B3FF005EAB5CA9DA
:1022B00058A956AB56B358B55CB55EB35EB15CAFCA
:1022C00058AF56B1FF0056A95EA95EAB5CAD5AB1DE
:1022D0005AB5FF0058AF56AD56AB58A95CA95EABD6
:1022E0005EAD5CAF58AF56B156B358B55CB55EB392
:1022F0005EB15CAFFF005EAD5CAF5CAF58AF56AD9A
:1023000056AB58A95CA95EAB5EB35CB558B556B385
:10231000FF008C119611991149AB4BA94FA951ABF4
:1023200051B34FB54BB549B349ABFF004DA94DB5BE
:10233000FF0049AB4BA94FA951AB51AD49B551B5C0
:10234000FF00303132333435363738394142434477
:1023500045460C0102030405060708090A0B0C0197
:1023600002030405060708090A0B00000100010129
:102370000001FF01FF00FFFF00FF447574636874F4
:10238000726F6E697820415652204F7363696C6C8E
:102390006F73636F706520436C6F636B2056000032
:1023A000456E74657220636F6D6D616E64202841A7
:1023B0002C422C432C442C462C482C4C2C4E2C507C
:1023C0002C532C542C56293A0000456E746572200B
:1023D0003220646967697420686F7572733A2020CF
:1023E0002000456E7465722032206469676974202C
:1023F0006D696E757465733A2000456E7465722060
:1024000032206469676974207365636F6E64733A20
:102410002000456E746572203220646967697420FB
:10242000796561723A2020202000456E7465722023
:1024300032206469676974206D6F6E74683A202079
:102440002000456E746572203220646967697420CB
:102450006461793A20202020200043616C69627217
:102460006174696F6E205061747465726E20000033
:102470004E756D6572696320646973706C61792053
:1024800000004C4544200000566572626F73652061
:102490000000414D2F504D20000041565220436C0A
:1024A0006F636B204D617374657220004275726EAC
:1024B0002D696E2050726576656E74696F6E2000AE
:1024C00046617374204D6F64652000005265766527
:1024D000727365204D6F6465200052657175657378
:1024E000746564206D6F64652072657175697265CD
:1024F000732041565220636C6F636B204D6173747F
:102500006572204D6F646500416C6C204469676999
:10251000747320646973706C6179200043616E6329
:10252000656C206F722054696D656F7574004E6F15
:102530007420456E746572696E672044656D6F2006
:102540004D6F646500000D0A00004F6E00004F667D
:1025500066004A616E1F4665621C4D61721F4170C4
:10256000721E4D61791F4A756E1E4A756C1F41754A
:10257000671F5365701E4F63741F4E6F761E446550
:10258000631F447574636874726F6E6978204F734B
:1025900063696C6C6F73636F706520436C6F636B02
:1025A0002048656C703A0D0A413A20546F67676C99
:1025B00065204D617374657220436C6F636B20629C
:1025C00065747765656E2041565220616E642052B5
:1025D00054430D0A423A20546F67676C6520427578
:1025E000726E2D696E2070726576656E74696F6E9D
:1025F0000D0A433A20446973706C61792043616C21
:102600006962726174696F6E207061747465726E54
:102610000D0A443A204368616E6765204461746521
:102620000D0A463A20546F67676C6520416C6C2038
:1026300044696769747320446973706C61790D0A29
:102640004C3A20546F67676C65204C454420626C9F
:10265000696E6B696E670D0A4E3A20546F67676C3E
:1026600065204E756D6572696320446973706C6195
:1026700079200D0A503A20546F67676C6520414DF0
:102680002F504D200D0A533A20446973706C6179C4
:1026900020537461747573200D0A543A20436861A5
:1026A0006E67652054696D650D0A563A20546F6750
:1026B000676C6520566572626F7365204F75747024
:1026C00075740D0A0000E0EBF5E1E0930A01F09368
:1026D0000B010895E6E0F6E1E0930A01F0930B01A7
:1026E00008950C850023D9F50E94C20636C00C85DA
:1026F0000023A9F10E94C20630C00F85002379F59E
:102700000E94E5062AC00F85002349F10E94E506D4
:1027100024C00FA1002319F50E9416071EC00FA1A7
:102720000023E9F00E94160718C00D850023B9F4B4
:102730000E94D50612C00D85002389F00E94D5069F
:102740000CC00B85002361F00E944B0606C00B8570
:10275000002331F40E944B0600C00E94460400C0D2
:10276000089509A10023E1F30E940C07F6CF09A107
:102770000023B1F70E940C07F0CF0E85002381F3F0
:102780000E94A506EACF0E85002351F70E94A506F8
:10279000E4CF0DA1002321F30E947C06DECF0DA122
:1027A0000023F1F60E947C06D8CF0EA10023C1F2CF
:1027B0000E949406D2CF0EA1002391F60E949406A7
:1027C000CCCF09A50195039509A7EAE1F3E1E093D0
:1027D0000001F09301010FA000FC0895EAEAF4E182
:1027E000E0930201F093030108950895F98E08958E
:1027F0000E94980708950E948C0708950E948307FD
:1028000008950E947707089501E00CA70E946313C2
:10281000C0DFCBDF96DFEAE9F9E20E948504EAE156
:10282000FAE20E9485040E9471130E948913E8E471
:10283000FAE20E9485040E948F13EAE6FAE20E94FF
:1028400085040E947D130E947713E8E8FAE20E9453
:1028500085040E948313EAEAFAE20E948504ECEC04
:10286000FAE20E9485040E947D130E9469040E947E
:1028700089130E9469040E9483130E9469040E94C4
:102880008F130E9471130E9469040E948F130E948B
:1028900077130E9469040E9489130E9471130E9499
:1028A00069040E948F130E9483130E9477130E9471
:1028B00069040E949513E8EEFAE20E9489040E94DE
:1028C0009B13E2E0FBE20E9489040E94A713E6E169
:1028D000FBE20E9489040E94A113E0E3FBE20E9454
:1028E00089040E94C313E2E4FBE20E9489040E946F
:1028F000CF13E4E7FBE20E9489040E947F040E9458
:10290000C913E6E8FBE20E9489040E94DB13EAE9AE
:10291000FBE20E9489040E94CF13ECEAFBE20E94D2
:1029200089040E947F040E946F0609E00CA70E94A0
:102930000114EAEEFBE20E9489040E947F0403E096
:102940000CA70E94FE130E94FB13ECE3FCE20E9422
:1029500089040E947F0401E10CA70E94F8130E94E1
:10296000E113ECE8FCE20E94890405E00CA70E9458
:10297000E1130E94F613EAEAFCE20E9489040E9435
:102980007F04FCA60E94F513EAE0FDE20E948504A4
:102990000E946A130E94DE000895546869732064DF
:1029A000656D6F206D6F64652073686F777320733A
:1029B0006F6D65206F662074686520636170616269
:1029C000696C6974696573206F662074686520445A
:1029D0007574636874726F6E69780D0A415652207F
:1029E0004F7363696C6C6F73636F706520436C6FBA
:1029F000636B2E20497420707265736572766573FF
:102A000020746865207374617465206F6620796F27
:102A1000757220636C6F636B2E0048657265206170
:102A2000726520736F6D65206F6620746865204342
:102A30006C6F636B20446973706C6179732073757C
:102A400070706F7274656400416E616C6F672043D3
:102A50006C6F636B2077697468206D696E696D6156
:102A60006C206469676974730000416E616C6F6704
:102A700020436C6F636B207769746820616C6C20F5
:102A80006469676974730000416464207468652038
:102A9000323420686F757273206E756D657269636C
:102AA00020646973706C617900004F722061646406
:102AB0002074686520414D2F504D206E756D6572F4
:102AC000696320646973706C617900004D697820D6
:102AD000616E64204D6174636820617320796F7545
:102AE00020706C65617365005475726E2074686542
:102AF000204C454420626C696E6B696E67206F667E
:102B00006600416E64207475726E20697420626183
:102B1000636B206F6E005475726E206F6E20436180
:102B20006C6962726174696F6E204D6F646500003C
:102B30005475726E206974206261636B206F6666E3
:102B4000000054686520274127206F6E2074686557
:102B50002073636F7065206D65616E7320415652FE
:102B600020436C6F636B204D6173746572204D6FF1
:102B7000646500004D616B652054696D6520676F69
:102B80002066617374004D616B652054696D65202A
:102B9000676F206E6F726D616C004D616B652054C4
:102BA000696D6520676F206261636B004D616B65C5
:102BB0002054696D6520676F206261636B206661D8
:102BC00073742100566572626F7365206F7574703F
:102BD0007574206973206F6E65206F6620796F753C
:102BE00072206F7074696F6E730054686520626C38
:102BF000696E6B696E67204220776F756C6420691F
:102C00006E6469636174652061206C6F7720525433
:102C100043206261636B75702062617474657279C0
:102C20002C20627574206E6F772069742773206A78
:102C300075737420612064656D6F0000546869735A
:102C400020626C696E6B696E67205020696E6469E2
:102C500063617465732074686174207468652031E1
:102C600020505053207369676E616C206973206D2A
:102C7000697373696E672E20416761696E2C206AE3
:102C800075737420612064656D6F000057696C6C0A
:102C900020746869732067657420796F757220618C
:102CA0007474656E74696F6E3F004275726E206950
:102CB0006E2070726576656E74696F6E206D6F76CA
:102CC00065732074686520646973706C6179206134
:102CD0002074696E79206269742C206E6F726D6148
:102CE0006C6C792065766572792035206D696E751A
:102CF00074657320627574206865726520657665F9
:102D00007279207365636F6E6400576520686F7019
:102D10006520796F7520656E6A6F796564207468C7
:102D200069732064656D6F2E205468616E6B207925
:102D30006F7520666F72207573696E67207468699D
:102D40007320447574636874726F6E697820436C85
:042D50006F636B0042
:00000001FF
